:1000000083160330850086018312910194019F01BC
:10001000BA2882073F3430345B344F3466346D3451
:100020007D3407347F346F346E343F343E340034D3
:1000300038343F346D3479340034FF340C088F0089
:1000400002300F06031D27280130900008000330FE
:100050000F06031D2E2802309000080004300F0602
:10006000031D352803309000080005300F06031DDE
:100070003C281108900008008F038F038F038F0323
:1000800020288D018E010C088F008F0A8F0B4928C4
:1000900008008D0A0A300D06031D46288E0A8D01C0
:1000A000462860309B00000000009A0B532805187A
:1000B0005D281F109B0B532808001F185A28940A0C
:1000C000141D8C03043093009F141F145A28003011
:1000D0000E0603197A280E08092086005120860191
:1000E00051200D0809208600512086015120512001
:1000F000512008000D08092086007628403086002F
:100100009A209A20063086009A209A209A209A20D7
:100110000D30920086019A20120809208600FF30D7
:1001200006060319BA28920A9A209A208A280A30C9
:1001300092008A2800009A0B9A289B0B9A280800A4
:1001400001301006031DA72880308600B028023039
:100150001006031DAE28C0308600B028E0308600AF
:100160000A309C0000009A0BB2289B0BB2289C0B13
:10017000B228080016308C00910A043011060319C9
:10018000D928412067209F1CBC28930BBC289401D0
:1001900000300C060319972801300C0603197E283D
:1001A0001E20A020412067208C03900BD2289F1096
:0801B000BC289101910AC1284D
:00000001FF
